:100000000C94FA000C9420010C9420010C94200113
:100010000C9420010C9420010C9420010C942001DC
:100020000C9420010C9420010C9420010C942001CC
:100030000C9420010C9420010C9420010C942001BC
:100040000C9465080C9420010C9420010C94200160
:100050000C9420010C9420010C9420010C9420019C
:100060000C9420010C948C020C9420010C9420011F
:100070000C9420010C9420010C9420010C9420017C
:100080000C9420010C9420010C9420010C9420016C
:100090000C9420010C9420010C9420010C9420015C
:1000A0000C9420010C9420010C9420010C94640306
:1000B0000C9420010C9420010C9420010C9420013C
:1000C0000C9420010C9420010C9420010C9420012C
:1000D0000C9420010C9420010C9420010C9420011C
:1000E0000C9420010C9420010C9420010C9420010C
:1000F0000C9420010C9420010C9420010C942001FC
:100100000C9420010C9420010C9420010C942001EB
:100110000C9420010C9420010C9420010C942001DB
:100120000C9420010C9420010C9420010C942001CB
:100130000C9420010C9420010C9420010C942001BB
:100140000C9420010C9420010C9420010C942001AB
:100150000C9420010C9420010C9420010C94220199
:100160000C9420010C9420010C9420010C9420018B
:100170000C9420010C9420010C9420010C9420017B
:100180000C9420010C9420010C9420010C9420016B
:100190000C9420010C9420010C9420010C9420015B
:1001A0000C9420010C9420010C9420010C9420014B
:1001B0000C9420010C9420010C9420010C9420013B
:1001C0000C9420010C9420010C9420010C9420012B
:1001D0000C9420010C9420010C9420010C9420011B
:1001E0000C9420010C9420010C9420010C9420010B
:1001F0000C94200111241FBECFEFDFE3DEBFCDBF83
:1002000000E00CBF18BE19BE1ABE1BBE10E2A0E073
:10021000B0E2EEE8F4E100E00BBF02C007900D92FF
:10022000AC3EB107D9F71BBE13E2ACEEB0E201C0A1
:100230001D92AF36B107E1F70E94F6070C94450A0C
:100240000C9450031F920F920FB60F9208B60F92A4
:100250000BB60F92112418BE1BBE8F939F93EF9382
:10026000FF9388E0E0E6F6E086838091C309E091A1
:100270002120F0E0E050F04E8083809121208E31EB
:1002800028F4809121208F5F80932120809120206D
:1002900081508093202080912020882331F581E0B7
:1002A00080931E208091222090912320892B91F40D
:1002B0008091C0098F7B8093C00980E8E0E6F6E07A
:1002C000858382E080930009809101098061E0E0EC
:1002D000F9E081838091222090912320019771F48D
:1002E00080E1E0E6F6E0858309C0E0912120F0E0BE
:1002F000E050F04E8081E0ECF9E08383FF91EF91D4
:100300009F918F910F900BBE0F9008BE0F900FBE64
:100310000F901F90189580E090E2089580911E2024
:10032000089580911F20089520912220309123204C
:10033000C901089580911E20882319F081E08093DF
:100340001F200895E0ECF9E08DED808383E0818348
:100350000895E0E0F9E082E0808381E18183128208
:10036000138214821682178282E090E080A791A700
:1003700008958091EC20882329F40E94A90181E04E
:100380008093EC2089E58093C00983E0E0ECF9E0FC
:1003900081830895DF92EF92FF920F931F93DF9373
:1003A000CF930F92CDB7DEB7E82ED92EF62E8091DF
:1003B0001F20882311F482E057C08DE1861710F4C6
:1003C00081E052C010921F2010921E20842F90E0D6
:1003D000809322209093232060932020109221204C
:1003E0008091C00980648093C009442319F0413092
:1003F00029F51DC010920009809101098F7EE0E06F
:10040000F9E0818300E616E091E0F8019683998394
:100410000E94B90188E0F80185839981892F8A9526
:10042000F1F79683892F8A95F1F7958307C08DEDB3
:100430008093C00983E0E0ECF9E081838E2D9D2D4F
:100440009C01D90120E030E007C08D91F901E05016
:10045000F04E80832F5F3F4F2F15B8F3809100201F
:10046000E0ECF9E0838380E00F90CF91DF911F9162
:100470000F91FF90EF90DF900895FC016383089542
:10048000FC018381089581E00895DF93CF9300D02C
:10049000CDB7DEB79C01673010F091E019C0606302
:1004A000698334E0969587953A95E1F78A83822FA0
:1004B0008295807F8B83CE01019663E041E00E94AC
:1004C000CA01982F882321F480E1E0E6F6E08683D4
:1004D000892F2396CDBFDEBFCF91DF910895E0E64F
:1004E000F6E080EB818380E1858386E0818382E092
:1004F000858384E085830895E0E6F6E089E08183E2
:1005000098E0968381E08583E0E8F6E08FE08183E0
:1005100085E08583958308951F920F920FB60F9201
:1005200008B60F920BB60F92112418BE1BBE8F9304
:10053000EF93FF93E0915E218091A008F0E0E05AF4
:10054000FE4D808380915E21883250F4809133216A
:10055000883230F480915E218F5F80935E2102C0EB
:1005600010925E21809133218F5F80933321FF9120
:10057000EF918F910F900BBE0F9008BE0F900FBEA2
:100580000F901F90189580913321089580915D21DF
:10059000E82FF0E0E05AFE4DE081883220F48F5FD2
:1005A00080935D2102C010925D21809133218823C8
:1005B00029F0809133218150809333218E2F08952B
:1005C0009C018091A10885FFFCCF862F90E0E0E0A0
:1005D000F1E084A395A3C90120A7AA2797FDA095C0
:1005E000BA2F292F3A2F4B2F552721A7CD01AA2704
:1005F000BB2782A780912001806880A308959C0179
:100600008091A10885FFFCCFE0E0F1E0809104013A
:1006100085FDF6CF862F90E084A395A3C90120A77E
:10062000AA2797FDA095BA2F292F3A2F4B2F552790
:1006300021A7CD01AA27BB2782A78091200180682E
:1006400080A30895E0E0F1E084E080A311A280E1BE
:1006500082A38CE483A316A280EA84A788E085A7FE
:1006600016A6089510925D2110925E2110923321FA
:10067000E0EAF8E080E3838388E1848383E0858394
:1006800081E2868380EF87830895982F8091A10867
:1006900085FD02C081E008959093A00880E0089550
:1006A0001F920F920FB60F9208B60F92112418BE28
:1006B0008F9381E080936A238F910F9008BE0F90F3
:1006C0000FBE0F901F9018951F920F920FB60F92AA
:1006D00008B60F92112418BE00000F9008BE0F90AC
:1006E0000FBE0F901F90189583E880930001089526
:1006F000DF93CF930F920F92CDB7DEB7DC0140E0CE
:1007000050E03C9120E011968C911197F901E80F8F
:10071000F11DE983FA8389819A81880F991F880FD7
:10072000991F89839A8389819A8195958795959553
:10073000879589839A8389819A81FB01E40FF51F4C
:100740008083918312964E5F5F4F4C305105C9F6FE
:100750000F900F90CF91DF910895E0E0F6E01082C6
:1007600031E0318392E0918383E08483E0E2F6E03C
:1007700010821482E0E4F6E010829483918328E0F2
:100780002183E0E6F6E010823183918344E04183E7
:10079000218380E1818380E2818380E8818381E11C
:1007A0008483E0E8F6E010823183918341832183E2
:1007B000148208958BECE0E5F0E082838091500094
:1007C0008860809350008091510083FFFCCF82ECC1
:1007D000E0E5F0E0858380915000806180935000D7
:1007E0008091510084FFFCCF88ED84BF84E080932A
:1007F000400080915000809350000895E0E0F8E0C0
:1008000085E0808381E1818312821382148288EEE5
:1008100093E080A791A783EF8487168283E0878384
:100820000895CF93DF93FC01DB012130A1F021304B
:1008300020F0223009F06FC059C0EC0120E030E018
:1008400007C0FD01E20FF31F899180832F5F3F4FA7
:100850002417B8F360C09181969596959C938181F9
:1008600087FF02C0906C9C9381818295880F880FCE
:10087000807C908196959695892B11968C931197F3
:1008800093819695969512969C931297838187FFF4
:1008900004C0906C12969C93129783818295880F66
:1008A000880F807C928196959695892B13968C93D0
:1008B000139795819695969514969C931497858198
:1008C00087FF04C0906C14969C9314978581829541
:1008D000880F880F807C948196959695892B159624
:1008E0008C931597868116968C9315C080818C9376
:1008F000818111968C931197848112968C93129713
:10090000858113968C931397828114968C931497F8
:10091000838115968C93DF91CF910895DF92EF92AA
:10092000FF920F931F93DF93CF93CDB7DEB7A097BE
:10093000CDBFDEBFAC017B01D22E1A8290E308C08E
:100940008A81F701E80FF11D90838A818F5F8A8386
:100950008A818D15A8F38E010D5F1F4FCA01B80162
:1009600040E150E00E94BC09198298010AC08981C7
:10097000F901E80FF11D8081882331F089818F5FB3
:10098000898389818D3198F38981D816C8F089814E
:100990008823B1F089818A839E012D5F3F4F0DC06E
:1009A0008A819A81D701A80FB11DF901E90FF11DC4
:1009B00080818C938A8181508A838A81882381F700
:1009C000A096CDBFDEBFCF91DF911F910F91FF9019
:1009D000EF90DF90089560E001C06F5FE62FF0E0D8
:1009E000EC5CFF4D80818823C1F784E390E20E9494
:1009F000E00208951F93FC018081813609F463C0F1
:100A0000843651F08F3309F026C181818F3309F08C
:100A100022C10E94EB04A1C08BE38093ED2080E310
:100A20008093EE2088E78093EF2080E28093F0208F
:100A30008093F1208093F2208093F3208093F42020
:100A40008093F520809124208093F62080912520AA
:100A50008093F720809126208093F8208091272092
:100A60008093F92081818233D1F0833330F4803355
:100A700061F0813309F0EFC00DC08433D1F08433CD
:100A800098F0853309F0E7C019C080912820909133
:100A9000292058C080912A2090912B2053C080910A
:100AA0002C2090912D204EC080912E2090912F20AF
:100AB00049C0809130209091312044C080913220F3
:100AC000909133203FC08BE38093ED2080E38093AF
:100AD000EE2088E78093EF2080E28093F0208093DF
:100AE000F1208093F2208093F3208093F420809370
:100AF000F520809124208093F620809125208093FA
:100B0000F720809126208093F820809127208093E1
:100B1000F9208181823341F1833340F4803371F0D5
:100B20008133E8F48A3209F096C035C0843331F15C
:100B30008433F8F0853309F08EC025C08091D4222B
:100B40009091D52260EF70E240E150E00E94BC0934
:100B50008DEE90E26DE00E94E00280E07DC0809129
:100B6000D6229091D722EECF8091D8229091D9228F
:100B7000E9CF8091DA229091DB22E4CF8091DC22D0
:100B80009091DD22DFCF8091DE229091DF22DACFBB
:100B90001093ED2001C01AE00E9491018823C1F357
:100BA0008091D4229091D5226EEE70E240E124E053
:100BB0000E948E0410E21093F2208091D622909130
:100BC000D72263EF70E240E124E00E948E0410938C
:100BD000F7208091D8229091D92268EF70E240E10D
:100BE00024E00E948E041093FC208091DA229091E0
:100BF000DB226DEF70E240E124E00E948E0410934E
:100C000001218091DC229091DD2262E071E240E1DD
:100C100024E00E948E04109306218091DE229091A0
:100C2000DF2267E071E240E124E00E948E048091BF
:100C3000242080930B218091252080930C2180918A
:100C4000262080930D218091272080930E218DEE08
:100C500090E262E280CF81E01F910895EF92FF92CF
:100C60000F931F93FC018081843609F042C18BE30E
:100C70008093102190E290931121909312219093F0
:100C80001321909314219093152190931621909302
:100C9000172190931821809124208093192180910D
:100CA000252080931A218091262080931B218091FA
:100CB000272080931C218181823309F46AC0833309
:100CC00030F4803371F0813309F013C136C08433BE
:100CD00009F4B7C0843308F488C0853309F009C12A
:100CE000DDC0FA01E60FF11D9083CA0160E070E0FB
:100CF00040E150E00E949E087B018C0180E0E816F4
:100D000080E1F80680E0080780E0180708F0F1C0ED
:100D1000C70161E171E240E150E00E94BC0980E15D
:100D200091E26DE00E94E002C70160E00E9445028E
:100D3000E0922820F0922920AFC0FA01E60FF11DC1
:100D40009083CA0160E070E040E150E00E949E089C
:100D50007B018C0180E0E81680E1F80680E008075E
:100D600080E0180708F0C5C0C70161E171E240E109
:100D700050E00E94BC0980E191E26DE00E94E00237
:100D8000C70161E00E944502E0922A20F0922B20E8
:100D900083C0FA01E60FF11D9083CA0160E070E0A4
:100DA00040E150E00E949E087B018C0180E0E81643
:100DB00080E1F80680E0080780E0180708F099C095
:100DC000C70161E171E240E150E00E94BC0980E1AD
:100DD00091E26DE00E94E002C70162E00E944502DC
:100DE000E0922C20F0922D2057C0FA01E60FF11D61
:100DF0009083CA0160E070E040E150E00E949E08EC
:100E00007B018C0180E0E81680E1F80680E00807AD
:100E100080E0180708F06DC0C70161E171E240E1B0
:100E200050E00E94BC0980E191E26DE00E94E00286
:100E3000C70163E00E944502E0922E20F0922F202D
:100E40002BC0FA01E60FF11D9083CA0160E070E04B
:100E500040E150E00E949E087B018C0180E0E81692
:100E600080E1F80680E0080780E0180708F041C03C
:100E7000C70161E171E240E150E00E94BC0980E1FC
:100E800091E26DE00E94E002C70164E00E94450229
:100E9000E0923020F092312080E02CC0FA01E60F81
:100EA000F11D9083CA0160E070E040E150E00E94D3
:100EB0009E087B018C0180E0E81680E1F80680E066
:100EC000080780E01807A8F4C70161E171E240E17A
:100ED00050E00E94BC0980E191E26DE00E94E002D6
:100EE000C70165E00E944502E0923220F092332073
:100EF000D3CF81E01F910F91FF90EF9008951F9342
:100F0000182F8D3021F08A3011F00E944503809116
:100F100031219091322181309105B9F081309105D4
:100F200038F08230910501F1039709F054C033C0C5
:100F3000109224211D3009F452C01A3009F44FC018
:100F400010932F2181E090E00AC01D3009F443C0C6
:100F50001A3009F440C01093302182E090E0809371
:100F600031219093322140C0103291F01D3011F0A8
:100F70001A3021F48FE291E20E94FA0484E290E2B6
:100F800064E00E94E00210923121109232212CC0C4
:100F900083E090E0E4CF1D3011F01A3079F4109224
:100FA0003121109232218FE291E26091242145E2B9
:100FB00051E20E942E068823B9F011C080912421AD
:100FC0008A3090F4E82FF0E0EB5DFE4D10838F5FE8
:100FD0008093242109C0109231211092322184E2A1
:100FE00090E264E00E94E0021F910895FF920F9347
:100FF0001F93DF93CF93CDB7DEB72C97CDBFDEBF66
:10100000CE0101968093892190938A210E94AD039D
:10101000E0E0F6E012E0158381E085830E94DA03C8
:101020000E9432030E94220388ED84BF80918000D9
:101030008D7F80938000E0E4F6E015838091A2002C
:101040008560E0EAF0E082830E946F020E947C02E9
:10105000789484E690E020E233E0F9013197F1F7EB
:101060000197D9F70E94FE0383E880930001E0E036
:10107000F6E082E0868381E0868384E290E264E0A9
:101080000E94E00200E016E0FF24F3940E94C302F5
:10109000882321F00E94C6020E947F070E948E01D1
:1010A000882351F00E949401892B31F40E948B0116
:1010B00064ED72E20E9478030E949A0180916A2393
:1010C000882321F3F801F582E1CF1F920F920FB62A
:1010D0000F9208B60F9209B60F920BB60F92112419
:1010E00018BE19BE1BBE2F933F934F935F936F9310
:1010F0007F938F939F93AF93BF93EF93FF938091D1
:10110000892190918A216CE040E00E94CA01FF9100
:10111000EF91BF91AF919F918F917F916F915F916F
:101120004F913F912F910F900BBE0F9009BE0F90E2
:1011300008BE0F900FBE0F901F9018953F924F92D0
:101140005F926F927F928F929F92AF92BF92CF9257
:10115000DF92EF92FF920F931F93CF93DF93EC01F7
:101160002B016A016115710519F0FB0180839183E0
:10117000C114D10449F0C6010297839728F020E0FA
:1011800030E040E050E0DCC0A9908A2D90E00E9461
:10119000B409892BC9F7FDE2AF1621F4A9903324D5
:1011A000339405C08BE2A81609F4A9903324C11426
:1011B000D10421F0E0E1CE16D10411F5F0E3AF1631
:1011C00069F48881883711F0883541F4A980229626
:1011D00082E0382A20E1C22ED12C12C0C114D104E1
:1011E00079F4E0E3AE1659F199E9E92E99E9F92E7F
:1011F00099E9092F99E1192F8AE0C82ED12C3AC01C
:10120000FAE0CF16D10491F080E1C816D10429F09C
:10121000E8E0CE16D104F9F415C0BFEFEB2EBFEF16
:10122000FB2EBFEF0B2FBFE01B2F24C0A9E9EA2E36
:10123000A9E9FA2EA9E90A2FA9E11A2F1BC0F8E0A3
:10124000CF2ED12CEFEFEE2EEFEFFE2EEFEF0E2F85
:10125000EFE11E2F0FC09601442737FD4095542F14
:101260006FEF7FEF8FEF9FEF0E94230AC901DA0132
:101270007C018D0120E030E040E050E060E036018C
:10128000882477FC8094982C70EDB72EBA0CF9E086
:10129000FB1570F48A2D81548A3118F499ECB92E1B
:1012A00006C08A2D81568A3148F589EAB82EBA0CD3
:1012B0008B2D90E08C159D050CF56F3FE9F0E21643
:1012C000F30604071507B8F0CA01B901A401930198
:1012D0000E94F0099B01AC018B2D90E0A0E0B0E0F2
:1012E000280F391F4A1F5B1F281739074A075B075A
:1012F00010F061E001C06FEFA990C6CF4114510416
:1013000051F0662311F0219703C031FE04C02297EB
:10131000F201C083D18330FE07C0509540953095CF
:1013200021953F4F4F4F5F4F67FF0AC082E290E029
:1013300080936D2390936E232FEF3FEF4FEF5FEF7E
:10134000B901CA01DF91CF911F910F91FF90EF90EA
:10135000DF90CF90BF90AF909F908F907F906F90D5
:101360005F904F903F900895911127C0803219F0FF
:1013700089508550D0F70895FB019F01E8944230D1
:10138000C4F04532B4F44A3029F497FB1EF490952A
:1013900081959F4F642F77270E940F0A805D8A33C3
:1013A0000CF0895D8193CB010097A1F716F45DE203
:1013B00051931082C9010C94E00999278827089558
:1013C000DC01FC01672F71917723E1F7329704C0AC
:1013D0007C916D9370836291AE17BF07C8F3089537
:1013E000629FD001739FF001829FE00DF11D649F09
:1013F000E00DF11D929FF00D839FF00D749FF00D95
:10140000659FF00D9927729FB00DE11DF91F639F35
:10141000B00DE11DF91FBD01CF0111240895AA1BD4
:10142000BB1B51E107C0AA1FBB1FA617B70710F0CF
:10143000A61BB70B881F991F5A95A9F78095909501
:10144000BC01CD010895A1E21A2EAA1BBB1BFD0110
:101450000DC0AA1FBB1FEE1FFF1FA217B307E40793
:10146000F50720F0A21BB30BE40BF50B661F771FEB
:10147000881F991F1A9469F76095709580959095CB
:0E1480009B01AC01BD01CF010895F894FFCF90
:10148E00000000000000000000000000000000004E
:10149E00000000000000000000000000000001013C
:1014AE00000000000A0D3A3EFF07FF07FF07FF0787
:1014BE00FF07FF070A2A2A2A2056455253494F4E44
:1014CE002039392E3939202A2A2A0A202D20613C2A
:1014DE00302D353E3A20646973706C617920414439
:1014EE00432076616C75650A202D20643C302D35C5
:1014FE003E3A20646973706C6179204441432076D2
:10150E00616C75650A202D20643C302D353E203CE3
:10151E006865782076616C75653E3A207365742037
:10152E004441432076616C75650A202D20733C730F
:10153E007C6D3E3A2073796E632070657220736104
:10154E006D706C65207C206D6561737572656D655F
:10155E006E740A202D203F3F202020203A20536811
:0C156E006F7720696E666F200A3A3E001D
:00000001FF
